:020000020000FC
:0200000004C03A
:100004002F912F91A4C001E003BF03E00FBD00E1D5
:1000140007BB00E108BB04E005BB00E20BBFE0E660
:10002400FF2700240082E395EE31E1F70FE90DBFCD
:100034009FEF8FEF07D1122F207C09F44FC0212F9F
:10004400207F205D19F5212F2F7023FF10C02A5027
:10005400A1F4F8D0203240F4205AE22FFF27E038F0
:1000640018F42191FCD0FBCF2227F9D0FDCF205AE0
:10007400E22FFF272081F3D0DBCF2350C9F627E4FA
:10008400EED020E5ECD023E0EAD0D2CF2051C9F461
:10009400212F2F7023FF0FC02A5051F6D3D02032C6
:1000A40040F4205AE22FFF27E03818F4CBD02193F4
:1000B400FBCFC8D0BDCF205AE22FFF27C3D0208367
:1000C400B7CF205109F0B4CF2FB52D7F10FF226098
:1000D4002FBD1F701695139513BFAACF5FEE15FDA4
:1000E4005AEF14FF5695546E13FD6CC012FD3BC0BD
:1000F40027B3252327BB24B3252324BB212F237017
:1001040059F10FEF0ABF789415FD10C014FD07C014
:10011400B39BFECF0197D1F0B399FECFF9CFB49B37
:10012400FECF019799F0B499FECFF9CF14FD07C023
:10013400B19BFECF019751F0B199FECFF9CFB09B9F
:10014400FECF019719F0B099FECFF9CFFFCFB29B44
:10015400FECF9095809552C0509506B3052309F0C3
:1001640020957FD065CF11FF16C06CD0209515FF68
:100174005FCF14FD08C029BD2FB52F7C206210FF6E
:1001840020612FBD1AC026BF2FB52F73206810FF22
:1001940020642FBD12C010FD03C028B3252304C062
:1001A400509528B3252B509528BB15FF06C02FB5B5
:1001B40014FD2F7314FF2F7C2FBD509527B3252BCF
:1001C40027BB36CF509524B3252B236024BB212F86
:1001D400237001F115FD10C006E806B922E010FFF6
:1001E400206212FD206414FF239527B9369A49D062
:1001F4003699FDCF84B195B1222733D011FD03C0C8
:10020400992309F08FEF292F11FD29D0282F10FDF4
:1002140026D00ECF212F2073205391F03798222718
:1002240012FD20E428B915FD06C022E014FF239531
:1002340027B91E9A01C01E9822270000459B2FEF64
:1002440010D0F6CE48E001C041E01BD02227B2997D
:10025400FECF17D0303427954A95C9F7089548E062
:1002640001C041E00ED0B299FECF20FD05C0BA9A7C
:1002740030E63A95F1F7BA9804D026954A9599F75D
:1002840008953327B299089500003395D9F7B29BA6
:04029400FECFCCCEFF
:00000001FF
